:020000040000FA
:10000000680A0020150200001D0200001F02000007
:100010002102000023020000250200000000000071
:1000200000000000000000000000000027020000A7
:1000300029020000000000002B0200002D02000039
:100040002F0200002F0200006D0500002F020000AB
:100050002F020000000000002F0200002F0200000D
:100060002F0200002F0200002F0200002F020000CC
:100070002F0200002F0200002F0200002F020000BC
:100080002F0200002F0200002F0200002F020000AC
:100090002F0200002F0200002F0200002F0200009C
:1000A0002F0200002F0200000000000000000000EE
:1000B0002F0200002F0200000000000000000000DE
:1000C0000000000000000000000000000000000030
:1000D0000000000000000000000000000000000020
:1000E0000000000000000000000000000000000010
:1000F0000000000000000000000000000000000000
:1001000000000000000000000000000000000000EF
:1001100000000000000000000000000000000000DF
:1001200000000000000000000000000000000000CF
:1001300000000000000000000000000000000000BF
:1001400000000000000000000000000000000000AF
:10015000000000000000000000000000000000009F
:10016000000000000000000000000000000000008F
:10017000000000000000000000000000000000007F
:10018000000000000000000000000000000000006F
:10019000000000000000000000000000000000005F
:1001A000000000000000000000000000000000004F
:1001B000000000000000000000000000000000003F
:1001C000000000000000000000000000000000002F
:1001D000000000000000000000000000000000001F
:1001E000000000000000000000000000000000000F
:1001F00000000000000000000000000000000000FF
:10020000DFF80CD000F02AF8004800473109000060
:10021000680A00200648804706480047FEE7FEE7D8
:10022000FEE7FEE7FEE7FEE7FEE7FEE7FEE7FEE7A6
:10023000810200000102000040EA01039B0703D095
:1002400009E008C9121F08C0042AFAD203E011F815
:10025000013B00F8013B521EF9D27047064C074D96
:1002600006E0E06840F0010394E807009847103486
:10027000AC42F6D3FFF7C8FF180F0000380F00009C
:10028000F0B5A848A74B012600781B1D1A1D4FF09A
:10029000805106280BD11C78240708D11478C4F3A8
:1002A0000314032C06D0042C04D0052C02D00628FD
:1002B00007D011E0B1F824439B4DC4F304242C6013
:1002C00002E01C78240707D11478C4F30314032C2C
:1002D00002D1974D954C6C67D1F83051D1F844421A
:1002E000944FC4F342343C6006280CD11C78240798
:1002F00009D11478C4F30314032C04D18E4C27685D
:1003000027F0807727604FF080470024C7F80C4122
:10031000C7F81041874F3F1F3C60062807D11F7860
:100320003F0704D11778C7F30317032F02D006281D
:1003300008D01FE0DFF8FCC103270CF1640CCCF8F7
:10034000007007E01F783F0714D11778C7F3031731
:10035000032F0FD1DFF8E4C10527CCF80070774FE9
:1003600078373E60754F08373C600CF1040C3F272E
:10037000CCF80070724F3F68DFF8C8C1CCF800704D
:100380006F4F3F1D3F680CF1040CCCF800706C4FB0
:1003900008373F680CF1040CCCF80070684F0C373C
:1003A0003F680CF1040CCCF80070654F10373F68C3
:1003B0000CF1040CCCF80070614F14373F680CF15D
:1003C000040CCCF800705E4F18373F68DFF874C13A
:1003D0000CF1200CCCF80070594F1C373F680CF121
:1003E000040CCCF80070564F20373F680CF1040C19
:1003F000CCF80070524F24373F680CF1040CCCF855
:1004000000704F4F28373F680CF1040CCCF8007097
:100410004B4F2C373F680CF1040CCCF80070484F60
:1004200030373F68DFF81CC10CF1400CCCF800708D
:10043000434F34373F680CF1040CCCF80070404F48
:1004400038373F680CF1040CCCF800703C4F3C3757
:100450003F680CF1040CCCF80070394F40373F680E
:100460000CF1040CCCF80070DFF8DCC0FB27CCF8F2
:100470000070062813D11F783F0710D11778C7F3F3
:100480000317032F03D0042F01D0052F07D1D1F874
:100490005872DFF8B8C007F04F07CCF800702C484E
:1004A0000268D20702D06FF001020260062D08D167
:1004B000D1F83401062804D12648016841F480614E
:1004C00001604FF01021D1F80002002803DBD1F8C1
:1004D0000402002822DA204A166020480368002B14
:1004E000FCD01523C1F800320568002DFCD0C1F8FE
:1004F000043201680029FCD0146001680029FCD096
:10050000BFF34F8F0C48F0380168154A01F4E061E1
:1005100011430160BFF34F8F00BFFDE7124911483F
:100520000860F0BDE00F00F0403501400DF0ADBABD
:1005300000C007403C050040FCED00E010560040C4
:100540000404001020C5004018F50040E40E0040EF
:10055000000400403C17004004E5014000E4014075
:100560000400FA050090D003200000200149024851
:1005700000F036BC2402002000200040014A02495D
:1005800000F013B8A10800001C00002002E008C819
:10059000121F08C1002AFAD170477047002001E0FD
:1005A00001C1121F002AFBD170472DE9F041164608
:1005B0000F460446002503E03946B047641C6D1C15
:1005C00020780028F8D12846BDE8F08172B60948A5
:1005D0000068C00700D000BEBFF34F8F0548E43865
:1005E0000168054A01F4E06111430160BFF34F8FD8
:1005F00000BFFDE7F0ED00E00400FA050EB50021B4
:100600000091CDE901106A4644F20100FFF7DEFFD8
:100610000EBD10B58268C368934203D000F02DF977
:10062000002010BD052010BD29B112B1531E134288
:1006300003D0092070470E2070470160838000219D
:100640008160C1600846704710B58268C3689A1A15
:1006500083889A4203D800F01AF9002010BD0420C4
:1006600010BD000070B50A4E01460A48B578FFF784
:10067000D0FF04464DB10020B070711C0122C81D8E
:1006800000F0C4F908B1FFF7B9FF204670BD0000C3
:100690000800002048020020F0B5244E89B01F4613
:1006A0000D00044672603FD0A888296882B22048B5
:1006B000FFF7BAFF002835D1A889A96882B21C4883
:1006C0001030FFF7B1FF00282CD1202219496846CD
:1006D000FFF7B2FD60690690207C00B101208DF823
:1006E00014008DF81C70607C00B10E208DF8150090
:1006F000E0680290A0680390206801906068009014
:100700000A480D4A6946083000F060F9002809D10E
:10071000B0702068401C05D004490122491CC81D46
:1007200000F074F909B0F0BD0720FBE708000020D5
:1007300048020020F80E0000110D000010B501461F
:100740000C48FFF781FF040011D10B4800F0BCFA00
:1007500068B9094907480C39FFF75BFF38B9064902
:1007600001220C3901F1080000F053F9044620463B
:1007700010BD000058020020140000202DE9F041B7
:10078000064608680C46411C4FF0A0474FF0010593
:1007900006D005FA00F1C7F80815206800F069F9DD
:1007A0006068411C02D0002100F05AF93168A0694C
:1007B000C1F82405607D217D32680843C2F86C05CC
:1007C000D4E900123068C0F80C15C0F81425207D5B
:1007D000012815D1A068411C02D0002100F040F989
:1007E000E068411C05D08540C7F80855E06800F076
:1007F00040F9D4E902123068C0F80825C0F8101595
:10080000BDE8F0812DE9FC410646C0074FF0000528
:100810000ED0104F00240122385D009500231146B0
:10082000019500F0F9F8641C042CF4D300F01CF8D6
:10083000B0070DD5074E0024361D0022305D03237E
:1008400000951146019500F0E7F8641C042CF4D3E0
:10085000BDE8FC81EC0E00000249085C012100F0BB
:1008600012B90000EC0E000010B500242046FFF77E
:10087000F3FF641C042CF9D310BD826883881A40EE
:1008800003689A5C0A708168491C81607047C2687D
:1008900083881A4003689954C168491CC160704735
:1008A00010B50446C0B2FFF749FF204610BD000056
:1008B00070B50D46044600684FF4887100F0F3F8F7
:1008C0004FF49071206800F0EEF84FF492712068B8
:1008D00000F0E9F84FF4A271206800F0E4F8206815
:1008E0001249C0F8041320686907000B40B2090ED2
:1008F000002806DA00F00F0000F1E02080F8141D57
:1009000003E000F1E02080F8001420680121000BD2
:1009100040B200F01F0291404009800000F1E02049
:10092000C0F88012C0F8001170BD00001003020072
:100930008AB00120FFF766FF182216496846FFF7C4
:100940007BFC1548069015494FF48070CDE90701EE
:1009500009900723124A06A96846FFF79DFE08B1D1
:10096000FFF74CFE0FA0FFF709FE06A8FFF77AFE7F
:100970000028FAD19DF81800FFF7E0FE0028F9D111
:100980009DF81800712801D05128EED10CA0FFF776
:10099000F5FDFEE7D40E0000240000202401002015
:1009A000FD0C00000D0A55415254206578616D70B0
:1009B0006C6520737461727465642E0D0A0000000A
:1009C000200D0A45786974210D0A000070B50646AD
:1009D00004780C4888B0154640F82420094A086974
:1009E000121D42F8240020226846FFF725FC0494DB
:1009F0000DB1054A00E000226946301D00F064F8A0
:100A000008B070BD00000020B10D0000001D00F016
:100A100091B8001D00F010B970B541EA4201DDE95E
:100A200004564FF0A04441EA830141EA052104EB5A
:100A3000800041EA0641C0F8001770BD70B541EA78
:100A40004201DDE904564FF0A04441EA830141EA46
:100A5000052104EB800041EA0641C0F8001770BD93
:100A60001CB500220B46009211460192FFF7E6FFEB
:100A70001CBD1CB5002100910B46012201911146BD
:100A8000FFF7DCFF1CBD01224FF0A043824011B1F3
:100A9000C3F808257047C3F80C2570474058002854
:100AA00000D00120704708B5002242504058009005
:100AB00008BD0121B1EB507F01D10120704700201A
:100AC00070470020704700002DE9F04105461646AA
:100AD00000790F46154A00EBC00102EB810494F83F
:100AE000201011B10820BDE8F081114951F8201003
:100AF0002868FFF7E6FF08B11120F4E739462846D9
:100B0000FFF73CFE6660386920601EB1397F2846D9
:100B1000FFF7CEFE28680821C0F800150020A0616C
:100B2000E0610121606184F82010DCE724020020EC
:100B3000F40E00002DE9F05F044600790E4600EB4C
:100B4000C001DFF8F0A017460AEB81053046FFF739
:100B5000B0FFB0B168684FF000084FF4047910B1ED
:100B60002168C1F80893A8694FF0000B80B1E869CB
:100B700048B1686810B12068C0F804931120BDE83E
:100B8000F09F1020FBE7EF614FF001082E6102E0BB
:100B9000EE60C5E9067B00254FF488712068FFF7F9
:100BA00082FF4FF4A2712068FFF77DFF2068C0F834
:100BB0003465C0F838752068B8F1000F12D0D0F84D
:100BC000001241F02001C0F800122079D04600EB5D
:100BD000C0010AEB8100406838B12068C0F8049376
:100BE0002846CCE701210160EFE74FF4887A4FF403
:100BF000A27951462068FFF751FF07464946206811
:100C0000FFF74CFF06464FF492712068FFF746FF4E
:100C1000014647EA06000843EBD0227902EBC20303
:100C200008EB8302C2F818B001B10325002ED7D01B
:100C30000F25D5E7240200202DE9F04704460E4693
:100C40000079204900EBC00001EB800517463046D3
:100C5000FFF72FFF30B1204600F036F820B1112009
:100C6000BDE8F0871020FBE76F61AE604FF490762F
:100C7000002731462068FFF716FF4FF4AC78414655
:100C80002068FFF710FF2068AA686969C0F844254A
:100C9000C0F84815206801218160686878B9B146BC
:100CA00049462068FFF7FAFE064641462068FFF7EE
:100CB000F5FE0643F4D000B10F27002068613846E6
:100CC000CEE70000240200200079054900EBC000B7
:100CD00001EB80004069002800D00120704700002F
:100CE000240200201FB501238DF800308DF8081074
:100CF0000192D0E90012684690471FBD0178022991
:100D000001D0012902D14068FFF778BC704700008C
:100D10007CB50178244D81B301290BD002292BD158
:100D20008DF80010C068691C01900122C81DFFF7F2
:100D30006DFE2EE0406801781C48FFF785FC1B4CD7
:100D4000012618B18DF80060019006E0A068E16806
:100D5000814205D000208DF8000069686846884708
:100D6000A068E168081AA188884207D80E490122C4
:100D7000491CC81DFFF74AFE7CBD01E0AE70FBE7D1
:100D80000A4809491030FFF744FC30B103208DF8C0
:100D90000000696868468847EEE70349012201F1CF
:100DA0000800FFF736FEE7E70800002048020020B1
:100DB0001FB50A4601788DF8001041680191017A4B
:100DC0008DF80810C0680390044850F82210001FE6
:100DD00050F82220684690471FBD00000400002004
:100DE0002DE9FF410C464FF4927705463946FFF74F
:100DF00055FE0026C0B139462846FFF754FE0220B2
:100E00008DF80000D5F88004C5F880040390D5F86B
:100E10003C058DF80800E0680190A661E661D4E920
:100E200000126846904723E04FF4887739462846F9
:100E3000FFF734FEE0B139462846FFF734FED5F817
:100E40003C15A069884213D1E06960B1E268D5F829
:100E5000000220F02000C5F80002E069A0612069CE
:100E6000E661E06001E0A661E2682046FFF73AFF34
:100E70004FF4A27739462846FFF710FE60B1394695
:100E80002846FFF710FEA06930B1A661D5F83C15E1
:100E90002046E268FFF726FF4FF490773946284650
:100EA000FFF7FCFD002813D039462846FFF7FBFD6D
:100EB000606900280CD0D5F84C058DF800608DF8DD
:100EC0000800A06801906661D4E900126846904766
:100ED000BDE8FF81080000000600000005000000DA
:100EE00007000000000000000000D60111121314DA
:100EF0000D0E0F106D050000FFFFFFFFFFFFFFFF4E
:100F0000FFFFFFFFFFFFFFFF0000000000000000E9
:100F10000000D60107000000380F0000000000208C
:100F2000240000008C0500005C0F0000240000205D
:100F3000440A00009C0500000000000000000000C2
:100F40000000000000000000000000000020004041
:0C0F500000000000000000000090D00332
:0400000500000201F4
:00000001FF
